:020000040000FA
:0600000060283D300130D4
:08000800A000030EA100831209
:1000100005191028831601178312B2308100422877
:100020008316011383120B191C28AE17280A031913
:100030002E17AE192D283B28AE13AE192A282E1FD5
:100040003B28AE1A3B28A701A601A501A801AE01D5
:10005000AE164228F030AE0542282D152E13AE12F2
:100060002708AB002608AA002508A9002808AC002C
:10007000F030AE0542282E0DA80DA50DA60DA70D3A
:10008000AE1AAE0A8B100B11210E8300A00E200EAB
:02009000090065
:1000C000203084008001840A80300402031C6228EE
:1000D000392283160C30850587018312850187013B
:1000E0000730990000309A00103083168E0083127A
:1000F000603083168F0083120030831691009F00BA
:100100008312C83083168100831231309000003092
:1001100083168C00831210308B00BD1B9128851D27
:1001200082223D1BBE013D1BBF013D1F7722810185
:100130008E018F010B118B100B108C018B17B020CF
:100140002D19B2200B22B30BAD280310851903140F
:10015000BA0DF0303A0203197A21BD18AA229F285D
:100160006400080029083F3C0319BE282B082A0612
:1001700029062C02031D2D11031D08002D1101302D
:10018000B7008B132030370783169B001C141A0806
:100190008312A4001030370783169B001C141A0822
:1001A0008312A3000030370783169B001C141A0823
:1001B0008312A2008B1724082B02031D7429230825
:1001C0002A02031D7429013003303702031D16294A
:1001D00029083F3C0319002940302906E039031D56
:1001E000F6283F1FF6283F13AD1704296030290673
:1001F000E039031D04293F1B04293F17AD170429CB
:10020000AC1F3F13AC1B3F1780302906F039031D8C
:100210000D29BF1F0D29BF13AD1790302906F039E6
:10022000031D1629BF1B1629BF17AD17A91F742957
:10023000291B742922082906F039A91EE039031D5B
:100240007429220829050F3903194A290130370278
:10025000031D2F293E182F293E14AD174F220230BF
:100260003702031D3829BE183829BE14AD17512294
:1002700003303702031D41293E1941293E15AD17B0
:10028000532204303702031D4A29BE194A29BE15DC
:10029000AD175722290922050F3903197429013096
:1002A0003702031D58293E1C58293E10AD175B220A
:1002B00002303702031D6129BE1C6129BE10AD1733
:1002C0005D2203303702031D6A293E1D6A293E1153
:1002D000AD175F2204303702031D7329BE1D732939
:1002E000BE11AD1763227429B70A0530370203180F
:1002F0000800C128B601B3019630B4000130B50042
:100300000130B70085018701AD13EB21B020B30B9D
:10031000AC29031085190314BA0DF0303A02031901
:10032000DB29B40BAC2901303702031967220230F4
:10033000370203196B220330370203196F2204308E
:100340003702031973223708B6080319B6000319D8
:10035000AA29B6039630B4002D1D86292D11A91F98
:100360008629291B8629A91E29120F302905031960
:100370008629B9012918B90AA918B90A2919B90A87
:10038000A919B90AB9188629391986298B13203079
:100390003707BC002B08BB00192210303707BC0000
:1003A0002A08BB00192200303707BC002908BB000F
:1003B00019228B17E52185018701B70AB60105309F
:1003C0003702031C862977220800043037020319FC
:1003D0000800850187011430B90033300F1E8500F5
:1003E0000F1A8501FF300F1A87000F1E8701B020FA
:1003F0002D1DED292D11290A0319022AA91FED2906
:10040000291BED290F302905031DEB29B90BED2917
:10041000850187010800AD1F0800AD131030BC0036
:100420003E08BB0019223030BC003F08BB00192237
:1004300008003C088B1383169B001C141A088312B7
:100440008B173B02031908008B133B0883161C15FE
:100450009A0083123C0883169B0055309D00AA30F9
:100460009D009C1464009C18322A1C1183128B1767
:100470000800831600309B001C141A088312BD006C
:10048000831610309B001C141A088312BE008316BA
:1004900030309B001C141A088312BF000800851618
:1004A000080005160800BD18080085140800BD18CE
:1004B0000800051408008512080005120800BD1880
:1004C000080085100800BD18080005100800050880
:1004D000203A850008000508103A85000800050844
:1004E000023A850008000508013A850008003E1818
:1004F0008516BE180516BD1808003E198514BE19CC
:1005000005140800B601B301B4013D1C8A2A3D1050
:10051000BD148D2AC030BD053D143D083F39B600DD
:100520006400922A932A942A952A962A3330B41B7F
:100530008500B41F8501B30B902AB40B902A0310D9
:10054000B60CB608031D902A0030BC003D08BB0065
:1005500019220800BF1FB52A3F1B85103F1B051439
:100560003F1F85143F1F0510080085100510080067
:02057000080081
:084000000500000006000200AB
:02400E00CC33B1
:1042000001008100820084008800B100B200B40087
:10421000B800A100A200FF00FF00FF00FF00FF00A8
:104220000000010001000100010001000100010087
:10423000010001000100FF00FF00FF00FF00FF0080
:10424000010000000000000000000000000000006D
:10425000000000000000FF00FF00FF00FF00FF0063
:104260000000FF00FF00FF00FF00FF00FF00FF0055
:10427000FF00FF00FF00FF00FF00FF00FF00FF0046
:10428000FF00FF00FF00FF00FF00FF00FF00FF0036
:10429000FF00FF00FF00FF00FF00FF00FF00FF0026
:1042A000FF00FF00FF00FF00FF00FF00FF00FF0016
:1042B000FF00FF00FF00FF00FF00FF00FF00FF0006
:1042C000FF00FF00FF00FF00FF00FF00FF00FF00F6
:1042D000FF00FF00FF00FF00FF00FF00FF00FF00E6
:1042E000FF00FF00FF00FF00FF00FF00FF00FF00D6
:1042F000FF00FF00FF00FF00FF00FF00FF00DD00E8
:00000001FF
